:10000000830100308A000428203084002D3016201F
:1000100083010730B600F830B5002D30840035304C
:100020001A208301662F04068001840A040603193E
:1000300000341328F00024208000840A040870068D
:10004000031900341B28B500B61B2F28361B372890
:1000500036088A003508B50A0319B60A82008313E8
:10006000361883173508B50A84000008080082078F
:100070003F3406345B344F3466346D347D3407349A
:100080007F346F348207063479347934F9345C3440
:0400900050346F3445
:100DBA0083120313AA000511803E0C2F831203131A
:100DCA00051101300C270230EA2E83120313AA0000
:100DDA000430AB005330AC00AC0BF12EAB0BEF2E52
:100DEA00AA0BED2E0800831203130515042F2B08F6
:100DFA00B6002A08AA0A0319AB0A23200C272B08D3
:100E0A00B6002A082320003803190800FC2E831292
:100E1A000313AA002A0E0F39F0000608F0397004ED
:100E2A008600851585112A080F39F0000608F03961
:100E3A0070048600851585110D30AB00AB0B232F8E
:100E4A00080083120313AA0005152A0E0F39F000B1
:100E5A000608F03970048600851585112A080F39AD
:100E6A00F0000608F03970048600851585110D30EA
:100E7A00AB00AB0B3E2F08008312031305110F3092
:100E8A00EA2603308600851585110530EA26851580
:100E9A0085112130AA00AA0B502F8515851105301E
:100EAA00EA2602308600851585110D30AA00AA0BA4
:100EBA005C2F28300C2708300C270F300C270630FF
:100ECA000C2F8316031385018601073083129F00B6
:100EDA0086018501A101A10A872F07302002031884
:100EEA00862F20082D3E84008313000885000030D9
:100EFA008A002008422086000230EA268601A00ADB
:100F0A00722FA10A96302102A001031C722F07300A
:100F1A0020020318972F2008223E840083138001A1
:100F2A00A00A8C2F22080A3A031D9D2FA30AA201A8
:100F3A0023080A3A031DA42FA40AA301A201240824
:100F4A000A3A031DAC2FA50AA401A301A201250890
:100F5A000A3A031DB52FA60AA501A401A301A201FD
:100F6A0026080A3A031DBF2FA70AA601A501A40154
:100F7A00A301A20127080A3A031DCA2FA80AA7013A
:100F8A00A601A501A401A301A20128080A3A031D8A
:100F9A00D62FA90AA801A701A601A501A401A301A8
:100FAA00A201A101A10A0F3021020318F62FA00104
:100FBA00073020020318D72F20082D3E8400831300
:100FCA000008850000308A002008063C223E840082
:100FDA0083130008372086000230EA268601A00A19
:100FEA00DD2FA20A972F0134023404340834103456
:060FFA0040348034003495
:02400E0050FF61
:00000001FF
